:100000002E288001840AFF3E031D01282928A5010E
:10001000A400FF30A407031CA507031C29280330F4
:10002000A300DF3015200928A301E83EA200A309A0
:10003000FC30031C1E28A20703181B28A20700007F
:10004000A30F1B2822182428A21C282800002828D7
:10005000080083138312031300000800073099007F
:1000600007309900FE3083168500811383128501C5
:100070002030840040300120851A3F283E283E3041
:100080000505AA003E302A0203193F280530072043
:100090003E300505A101A0002108031D53282008BA
:1000A0002A02031954283F2802302A05A101A00082
:1000B00021082004031D5E281130A70004302A0502
:1000C000A101A00021082004031D68281030A7000A
:1000D00008302A05A101A00021082004031D722870
:1000E0002030A70010302A05A101A000210820041B
:1000F000031D7C282130A70020302A05A101A00083
:1001000021082004031D86280C30A70003012618AF
:100110000130013A03192610031D26143E3005054F
:10012000A101A00020083E3A210403199B289C202D
:10013000523007208E283F28D520271FD520271B87
:10014000D2202618D520261CD220001AD520001E29
:10015000D2208019D520801DD2200019D520001D65
:10016000D2208018D520801CD2200018D520001C59
:10017000D220A71AD520A71ED220271AD520271EA5
:10018000D220A719D520A71DD2202719D520271D99
:10019000D220A718D520A71CD2202718D520271C8D
:1001A000D2200800E320D8200800D820E32008004F
:1001B0006430A90000000000000000000000000002
:1001C000A90BDA2808002030A80000000430A9009C
:1001D000A90BE82805140130A900A90BED2805108A
:0601E000A80BE528080051
:02400E00C43FAD
:00000001FF
